:020000040000FA
:040000000000512883
:040004000034003490
:08000800F000030E8301F1007A
:100010000A08F2008A018C105B0803191E28DB1CF9
:10002000152805183728DB104A28051C3028DB0165
:100030009030D000D2000130D300D10051085302DB
:1000400003192528031832282B28500852020319B7
:100050004A28031832280130D00203183028D10270
:10006000DC0338280130D007031C3728D107DC0A0D
:100070005C0807393D2086004A28D90000308A00F4
:10008000590882079034103450344034603420349E
:10009000A034803472088A00710E8300F00E700E56
:1000A0000900D001D101D201D3011F30D4000330A7
:1000B000D5000330DB004130C000BD01C101C201E9
:1000C000C301C401C501C601C701C8012030B80081
:1000D0008312B901380884003908840783169B000D
:1000E0001C141A0883128000B90A0F303902031D4C
:1000F0006A284330B2004C30B3005330B40054305F
:10010000B5003030B6003230B000B1012930B8004F
:10011000B901BA01BB01BD0107309F0083160F3042
:100120008600FF30850083128316BE309200831252
:100130000F3092008316203099000430980083120B
:10014000903098008B170B1783168C1483128B1723
:100150008C1AAB28A8288B131A08BC008C123B18E9
:100160000429BA1BDA283008840031088407000803
:100170003C02031DC528B10A05303102031DC62803
:10018000B101B901FF30BA00A728B10138088400D5
:100190003908840700083C02031DD828B90A053035
:1001A0003902031DA728B101B901FF30BA00A72801
:1001B000B901A7283C08BA00FF30BB0000308A0014
:1001C0003A080F39EF20CD004D0803191229BD015F
:1001D000D801CD1FA728CD132808D800A728D900FB
:1001E00000308A0059088207003402348234003417
:1001F0000034003400340034003405340134003459
:100200000034003400340034D80803190929D80315
:10021000A728400884003D0884073C088000BD0AE8
:10022000CD0BA728BD01BB0101308A003A080F3968
:100230001C3E03188A0A820051282E292E292C29B7
:100240002C292C292C292C292C294C2942292C29D0
:100250002C292C292C292C29BA01A728BA014108BC
:10026000D2004208D30053085502031C3D29031D48
:10027000A728520854020318A7285508D300540889
:10028000D200A7284108A8000830D7002830D6009F
:100290000130BE00BA015D294108A9004208AA0048
:1002A0004308AB004408AC004508AD000930D70056
:1002B0002930D6000530BE00BA0156088400000877
:1002C00083169A008312570883169B009C111C15F5
:1002D00055309D00AA309D009C141C1183128C1F68
:1002E0006F298C13D70AD60ABE0B5D29B901BA0152
:0402F000BB01A7287F
:02400E00623F0F
:1042000000000000000000000000000000000000AE
:1042100000005600530049003000310020005300D8
:104220005400500052002000560031002E00300093
:04423000300030002A
:00000001FF
